:03000000023BC9F7
:0C3BC90078FFE4F6D8FD75816A023C101C
:100FA90020000A3C2E2E2E3E004950436F6E6E657E
:100FB90063745245510A004950436F6E6E656374FC
:100FC900000A49504E6F41434B210A003E432C56BB
:100FD9002C43432CC0E4E0EFF2E5F020D1E8EDEA40
:100FE900EEEC49500A003E432C4D41432C2530324A
:100FF90062583A25303262583A25303262583A25D9
:10100900303262583A25303262583A2530326258C5
:101019002C4D414320E0E4F0E5F10A003E432C5613
:1010290045522C20332E3220EEF2202573202573D1
:101039002CC2E5F0F1E8FF20495020ECEEE4F3EB97
:10104900FF0A0053657020303620323031320031CA
:10105900353A32313A3235003E432C4C442C505209
:101069004F473A2020202020202020202020202007
:101079002020202020202020202020202020202067
:101089002020202020202020202020202020202057
:101099002020202020202020202020202020202047
:1010A90020202020202020202CC4E0F2E020EFF096
:1010B900EEF8E8E2EAE828F4E0E9EB290A003E2A3A
:1010C9002C312CCEF1EDEEE2EDFBE520EFE0F0E086
:1010D900ECE5F2F0FB20F1E5F2E5E2EEE3EE20E8E3
:1010E900EDF2E5F0F4E5E9F1E00A003E412C41308A
:1010F900312C2562752E2562752E2562752E256285
:10110900752C495020E0E4F0E5F120E0E4E0EFF24D
:10111900E5F0E00A003E412C4130322C2562752E63
:101129002562752E2562752E2562752C495020E0A1
:10113900E4F0E5F120EEF1ED2E20F1E5F0E2E5F045
:10114900E00A003E412C4130332C2562752E256280
:10115900752E2562752E2562752C495020E0E4F024
:10116900E5F120F0E5E72E20F1E5F0E2E5F0E00A0F
:10117900003E412C4130342C2562752E2562752E96
:101189002562752E2562752CCCE0F1EAE020F1E5A7
:10119900F2E80A003E412C4130352C2562752E2596
:1011A90062752E2562752E2562752CD8EBFEE70A2D
:1011B900003E2A2C312CC4EEEF2E20EFE0F0E0ECBB
:1011C900E5F2F0FB20F1E5F2E5E2EEE3EE20E8EDF1
:1011D900F2E5F0F4E5E9F1E00A003E422C53303142
:1011E9002C2562752CC6E4E0F2FC20E7E0EFF0EE76
:1011F900F1E020F1EEE5E4E8EDE5EDE8FF20EEF2BF
:1012090020F1E5F0E2E5F0E00A003E422C533032ED
:101219002C2562752CCEE1ECE5ED20F120F1E5F00D
:10122900E2E5F0EEEC20E1E5E720EAE2E8F2E0EDC4
:10123900F6E8E90A003E422C5330332C2562752C1E
:10124900CFE5F0E5E7E0EFF3F1EA20EFF0E820EF92
:10125900EEF2E5F0E520F1E2FFE7E820F120F1E523
:10126900F0E2E5F0EEEC0A003E422C5330382C2532
:1012790062752CCCE5E4EBE5EDEDFBE92049502066
:10128900EAE0EDE0EB28E7E0E4E5F0E6EAE020E477
:10129900EE203520F1E5EA290A003E422C5330358B
:1012A9002C2562752CCAE0EDE0EB20F8E8F0EEEAB7
:1012B900EEE2E5F8E0F2E5EBFCEDEEE3EE20EEE13F
:1012C900ECE5EDE00A003E532C5330362C25303244
:1012D90062582530326258253032625825303262E0
:1012E90058253032625825303262582C4D414320FE
:1012F900E0E4F0E5F120F8E8F0EEEAEEE2E5F8E006
:10130900F2E5EBFCEDEEE3EE20EEE1ECE5EDE00AD3
:10131900003E454E440A000A44756D70582020204D
:10132900202030302030312030322030332030340A
:1013390020303520303620303720303820303920E1
:101349003041203042203043203044203045203085
:1013590046000A3A003A20000A000A44756D7044B2
:1013690020202020203030203031203032203033EE
:1013790020303420303520303620303720303820A6
:101389003039203041203042203043203044203051
:101399004520304600457272206B65790052642001
:1013A900656570726F6D0A005264204D454D0A00E3
:1013B900526420436F64650A00577269746520435B
:1013C9006F64650A0044656275674950204F4E0A8B
:1013D9000044656275674950204F46460A004465D6
:1013E90062756755736572204F6E0A0044656275B0
:1013F9006755736572204F46460A004465627567F2
:101409004D7367204F6E0A0044656275674D7367B7
:10141900204F46460A00436F6E666967206C6F630A
:101429006B210A00577220656570726F6D0A002082
:101439005361766520656570726F6D210A0045728A
:1014490072204D414321004C6F61643E3E002A00E9
:10145900CEF8E8E1EAE00A00202D20257528257557
:10146900290A003C4130313D003C4130323D003CCD
:101479004130333D003C4130343D003C4130353D45
:10148900003C21003C5330313D003C5330323D009B
:101499003C5330333D003C5330353D003C533038EC
:0814A9003D003C5330363D00CC
:06443900016700016500AF
:10449500C28E438910E4F58B758DB8D2ABD28E22CE
:03001B00023B396C
:103B3900C0E0C083C082C0D0C28E758B00758DB8BD
:103B490020060675A61E75A6E10565D202E5676021
:103B5900020567056AE56A540F7051E566D3940159
:103B690040021566D20EE56A543F7012D200906683
:103B79008EE0600A04F0E0D394B44002D206906665
:103B890087E0600204F0906104E0600214F090663E
:103B99008FE0D394014003E014F03005020568E595
:103BA90069D394644004D20680020569E564D3941C
:103BB9000140021564D28ED0D0D082D083D0E032B9
:10092100C291C290D2B5C20B7D027C007F071244F6
:100931001C8F25E525646060097D017F601243936A
:10094100D20BE4FDFC7F0B12441C8F25E52530E61C
:10095100097D04E4FF1243B7D20B7D017C007F07C0
:1009610012441C8F25E5257008FD7FFF124393D2A9
:100971000B300B03126000C288C2A8C2AA7589009D
:10098100123EF190633FE0B4FA06A3E064CE607BCF
:10099100E4F52574372525F582E43463F583E4F025
:1009A1000525E525B443EC90633F74FAF0A374CEBA
:1009B100F0A374CCF0906345740AF0E4A3F0A304AF
:1009C100F0A3F090633B74FFF0A3F0A3F0E4A3F075
:1009D1009063567403F0E4F525E5252401FFE43323
:1009E100FE74372525F582E43463F583E0FD124377
:1009F1006F0525E525C3944340DFE4F5A775A61EE1
:100A010075A6E1907FF0F0A3F080FE90634A740335
:100A1100F0A374CCF0E4906349F090668CF0A3F0FD
:100A21001235A2C2B51243DBC20612416ED20BC20D
:100A31000DC20C9065777408F09062B57424F0E4EF
:100A4100A3F090633FE09062B7F0906340E0906262
:100A5100B8F0906341E09062B9F0906342E0906237
:100A6100BAF0906343E09062BBF0906344E090621F
:100A7100BCF0756601E4906578F0C207C208C2094E
:100A8100C20A200B18AF25FE7D03123688E4FF123F
:100A91003A897E0F7FA9E4FBFDFC1231BA90668E84
:100AA100E060037401F0E4906104F0F5689065760C
:100AB100F0F56912449575A70775A61E75A6E1D2D2
:100AC100AFE4F569906104E070031214B190668F90
:100AD100E06401701D9080007410F09080A874FF94
:100AE100F0A3F0A3F0A3F0E490668FF0D20BC20C58
:100AF100C20D908008E0F52530E405D2077410F0AE
:100B0100E52530E508D2099080087420F0E525300C
:100B1100E608D2089080087440F0E568C394034069
:100B210019908002E4F0908001F0908000F0E56877
:100B310094064006E4F56812416E9080A0E07003CF
:100B4100123FE99080B8E07003123F6F9080D0E0CF
:100B51007003124112908000E070133007101232BE
:100B6100C1906332EFF0D3940040031200369080BD
:100B710002E07006908000E06005D205020AC2C260
:100B810005E4F568906104E06003020AC2200B12DB
:100B9100906579E0600C7E0F7FAB1234BAE490650A
:100BA10079F0300912122D73906332EFF0D3940073
:100BB1004005E0FF121F07200803020D46122BEC2F
:100BC100906332EFF07003020AC2906376E054BF83
:100BD100247F7003020CA1147003020C79240260BB
:100BE10003020CE8200B077E0F7FB21234BA200FEC
:100BF10003020D4690634EE07006906352E0606719
:100C0100906683E0FF90634EE0B50724906684E030
:100C1100FE90634FE0B50618906685E0FE90635044
:100C2100E0B5060C906686E0FE906351E06E603799
:100C3100906352E06F6003020D46906684E0FF907E
:100C41006353E06F6003020D46906685E0FF906399
:100C510054E06F6003020D46906686E0FF90635595
:100C6100E06F6003020D46C2039065787401F012D3
:100C710044D0756601020D4690668EE060037401F2
:100C8100F090667BE0FF906378E06F6003020D46B1
:100C910090667BE004F0E4F566906576F0020D461F
:100CA100300303020D46906345E07003020AC290CF
:100CB10062B4E06008906356741EF080069063563B
:100CC1007403F0123055D203E4F566906576F09026
:100CD100668704F0E490667AF0A3F0200B677E0F3C
:100CE1007FC01234BA805E90668EE060037401F0BA
:100CF100300352906376E020E74B906378E0FF90F9
:100D0100667AE0FE6F600D906682E07007EE146F08
:100D11007033801390667AE004F0906332E0FFD381
:100D2100940440031244CA9060007482F0A37401D9
:100D3100F0906378E0906002F07E607F007D0312A6
:100D41003CDC020AC2200303020E69E566706E12E2
:100D510044CDEF60237E647F76906477E02404FDC8
:100D6100123CDC906682E07009906356E0F5660201
:100D71000AC2E4F566020AC2906687E0D3943C4059
:100D81003C906682E070369062B4E0703090668785
:100D910004F01239D4E4906476F0A37412F09066F2
:100DA1007BE0906478F0A374FDF090610563A2018B
:100DB10090647A63A2017F121225E080981244BFE9
:100DC1008F25E525B401159060007483F0E4A3F04C
:100DD1007E607F007D02123CDC020AC2E525D394CD
:100DE10001401C9060007483F0A37401F0E5252498
:100DF100FEA3F07E607F007D03123CDC020AC2E5A7
:100E01006664016003020AC2906576E004F0200B7B
:100E1100077E0F7FCA1234BA906576E0FFD3940142
:100E2100400B906356E0941E5003E004F0EFC3942E
:100E310005400DC203E4906578F01244D0020AC265
:100E41007C667D8390634AE0FAA3E0FB7F02123E59
:100E51006D7E647F76906477E02404FD123CDC9023
:100E61006356E0F566020AC2E56664016003020AA0
:100E7100C2906578E014604624FE6042147003025B
:100E81000F5C24046003020AC2E4F568200F13908A
:100E910065787404F0906576E05401F0756601029E
:100EA1000AC29080027410F0E4906578F090657643
:100EB10004F075661290668374FFF0020AC29066B0
:100EC10083E07003020F469064767480F09064783A
:100ED1007401F0E4A3F0A304F0A37430F0A3747BD5
:100EE100F0E4F525747D2525F582E43464F58374F9
:100EF1007DF0747E2525F582E43464F583E4F0E524
:100F0100252407906477F07C667D8390634AE0FA3C
:100F1100A3E0FB7F02123E6D7E647F76E525240906
:100F2100FD123CDC906682E0601B123055D203E476
:100F3100F566906576F090668704F0E490667AF045
:100F4100A3F0020AC2300F07E4906578F0800690A2
:100F510065787404F0756612020AC29080027410FA
:100F6100F0756603906576E06401FFF09065787432
:100F710001F0EF7019906352E06013FCA3E0FDA350
:100F8100E0FEA3E0FF906683122372020AC290631F
:100F91004EE0FCA3E0FDA3E0FEA3E0FF9066831218
:070FA1002372020AC280FE68
:010FA8002226
:10003600906377E0B444047F0180027F009063768A
:10004600E0B447047E0180027E00EE5F604A906362
:100056003FE0906378F0906340E0906379F09063BE
:1000660041E090637AF0906342E090637BF09063A6
:1000760043E090637CF0906344E090637DF090638E
:10008600777452F09062AE63A2019080A863A201D9
:100096007F061225E0020917906332E0C3940850E8
:1000A6000302092090633FE0FF906378E06F6003EE
:1000B600020920906340E0FF906379E06F600302DD
:1000C6000920906341E0FF90637AE06F60030209C4
:1000D60020906342E0FF90637BE06F60030209209B
:1000E600906343E0FF90637CE06F60030209209019
:1000F6006344E0FF90637DE06F6003020920906334
:1001060077E06444701A9080A8E0B4FF139062AE62
:1001160063A2019080A863A2017F061225E08010E9
:100126009062B2E09080ACF09062B3E09080ADF067
:1001360090668EE060037401F090668F7464F090B0
:1001460063777452F0906376E0646D60030202BADE
:100156007BFF7A0F79D51218DF7BFF7A0F79EF9044
:10016600633FE0F52EA3E0F52FA3E0F530A3E0F51D
:1001760031A3E0F532A3E0F5331218DF752EFF75D3
:100186002F1075304C7531FF7532107533587BFF63
:100196007A1079251218DF7BFF7A1079611218DF41
:1001A6007BFF7A1079C71218DF7BFF7A1079F490FB
:1001B6006345E0F52EA3E0F52FA3E0F530A3E0F5C7
:1001C600311218DF7BFF7A11791E90634EE0F52E0F
:1001D600A3E0F52FA3E0F530A3E0F5311218DF7B9D
:1001E600FF7A11794C906352E0F52EA3E0F52FA328
:1001F600E0F530A3E0F5311218DF7BFF7A11797A4A
:1002060090633BE0F52EA3E0F52FA3E0F530A3E0E5
:10021600F5311218DF7BFF7A11799D906337E0F58F
:100226002EA3E0F52FA3E0F530A3E0F5311218DF99
:100236007BFF7A1179BA1218DF7BFF7A1179E3A274
:100246000FE433F52E1218DF7BFF7A1279139066CE
:1002560082E0F52E1218DF7BFF7A12793E90668EC9
:10026600E0F52E1218DF7BFF7A1279719062B4E006
:10027600F52E1218DF7BFF7A1279A3A201E433F57B
:100286002E1218DF7BFF7A1279CF90667CE0F52E6E
:10029600A3E0F52FA3E0F530A3E0F531A3E0F532B6
:1002A600A3E0F5331218DF1233C57BFF7A13791AF0
:1002B6001218DF22906376E0644C70737E137F2001
:1002C600FBFDFC1231BA90637EE0F526A3E0F5272C
:1002D600E4F529E526906380F0A3E527F07E137FF9
:1002E6005B7C637D807B021231BAE4F52885278228
:1002F600852683E0FF74802528F582E43463F58340
:10030600EFF00527E527700205260528E528B41035
:10031600DC7E137F5E7C637D807B101231BA0529FB
:10032600E529C3941040AC7E137F611234BA229043
:100336006376E0646C7060F52A7E137F63FBFDFCD8
:100346001231BAE4F529E4906380F0A3E52AF07E41
:10035600137F5B7C637D807B021231BAE4F528A8AB
:100366002AE6FF74802528F582E43463F583EFF0EE
:10037600052A0528E528B410E67E137F5E7C637D9A
:10038600807B101231BA0529E529C3940840B77E4F
:10039600137F611234BA22906376E0644B7061F584
:1003A6002874682528F582E43463F583E0603274A6
:1003B600682528F582E43463F583E0F460237468E5
:1003C6002528F582E43463F583E0FF747E2528F55D
:1003D60082E43463F583E0B507100528E528B40800
:1003E600C09061047432F00209179063767421F0AC
:1003F600300B030209177E137F9E1234BA020917C7
:10040600906376E0B4521A200B077E137FA612344F
:10041600BA9063767472F07E637F767D08123C55DF
:1004260022906376E064497045200B077E137FB106
:100436001234BA90637EE0F526A3E0F527E4F528AA
:10044600852782852683E0FF74802528F582E4349B
:1004560063F583EFF00527E527700205260528E5F5
:1004660028B480DC7E637F767D8A123C55229063B9
:1004760076E064437046200B077E137FB91234BAC8
:1004860090637EE0F526A3E0F527E4F5288527822C
:10049600852683E493FF74802528F582E43463F58A
:1004A60083EFF00527E527700205260528E528B421
:1004B60080DB7E637F767D8A123C5522906376E0F0
:1004C600645A7053200B077E137FC21234BA9063AE
:1004D6007EE0F526A3E0F5277C637D807B80AF2751
:1004E600AE26124314E4F528852782852683E493F5
:1004F600FF74802528F582E43463F583EFF0052741
:10050600E527700205260528E528B480DB7E637F93
:10051600767D8A123C5522906376E064446003023D
:1005260005AE90637EE0FF64447003020917EFB4E2
:10053600310CC20B7E137FCE1234BA0209179063B8
:100546007EE0B4300CD20B7E137FDA1234BA020985
:100556001790637EE0B4320CD20C7E137FE7123420
:10056600BA02091790637EE0B4330CC20C7E137F87
:10057600F51234BA02091790637EE0B4340CD20D3A
:100586007E147F041234BA02091790637EE0B435F4
:100596000CC20D7E147F111234BA02091790637EC5
:1005A600E0FF12001E020917906104E07013200B91
:1005B600077E147F1F1234BA9063767421F0020905
:1005C600179061047432F0906376E0FFB45104C270
:1005D600AF80FEEF64577045200B077E147F2D1207
:1005E60034BA90637FE0906332F0E4F5289063328A
:1005F600E0FFE528C39F400302091774802528F50C
:1006060082E43463F583E0FF90637EE0252824AD21
:10061600F582E43461F583EFF0052880D0906376A7
:10062600E0645360030206D1200B077E147F381264
:1006360034BA90633FE0FF9061B6E06F703C906320
:1006460040E0FF9061B7E06F7030906341E0FF904B
:1006560061B8E0B50724906342E0FF9061B9E0B568
:100666000718906343E0FF9061BAE0B5070C90630A
:1006760044E0FF9061BBE06F60169063767421F0F2
:10068600300B030209177E147F471234BA0209178A
:10069600E4F528E4F569AF28FE74AD2528F582E473
:1006A6003461F583E0FD12436F0528E528C394FE07
:1006B60040E1C2AFE4907FF0F0A3F0907FFD74AA12
:1006C600F0A374FFF0A37455F080FE906376E064A7
:1006D6004F705A90637EE0F526A3E0F527E527459F
:1006E60026700A200B077E147F501234BA200B079F
:1006F6007E147F571234BAE4F52874802528F582D3
:10070600E43463F583E0852782852683F00527E5B3
:1007160027700205260528E528B480DE90668DE060
:100726002480F090668CE03400F00209179063761E
:10073600E06445707490637EE0FEA3E0FF907FF076
:10074600EEF0A3EFF0D39400EE94044038907FF0DF
:10075600E0FEA3E0FF90668CE0FCA3E0FD9FEC9E2C
:100766004023E42FFFEE3401FED3ED9FEC9E50159F
:10077600C2AF907FFD74AAF0A374FFF0A37455F086
:10078600E4F5A780FE7E147F591234BA7BFF7A14F3
:100796007961907FF0E0F52EA3E0F52F90668CE06E
:1007A600F530A3E0F5311218DF906376E0646560FA
:1007B6000302092090637EE0FFA3E0907FF0CFF074
:1007C600A3EFF0E4F526F527D3907FF1E095279087
:1007D6007FF0E095264020E4F5692527FFE52634DD
:1007E60001FE852782852683E0FD12436F0527E5F6
:1007F600277002052680D17E147F6C123D63EF4E72
:100806006020120003906345EFF0120003906346E8
:10081600EFF0120003906347EFF012000390634875
:10082600EFF07E147F72123D63EF4E6020120003DC
:1008360090634EEFF012000390634FEFF012000347
:10084600906350EFF0120003906351EFF07E147F37
:1008560078123D63EF4E6020120003906352EFF072
:10086600120003906353EFF0120003906354EFF00D
:10087600120003906355EFF07E147F7E123D63EF06
:100886004E602012000390633BEFF012000390636A
:100896003CEFF012000390633DEFF012000390630B
:1008A6003EEFF07E147F84123D63EF4E602012000F
:1008B60003906337EFF0120003906338EFF01200F5
:1008C60003906339EFF012000390633AEFF0E4F51A
:1008D60028E4F569E5282401FFE433FE743725286A
:1008E600F582E43463F583E0FD12436F0528E528BD
:1008F600C3944340DCC2AFE4907FF0F0A3F0907F56
:10090600FD74AAF0A374FFF0A37455F0E4F5A78074
:0A091600FE7E637F767D08123C55DB
:0109200022B4
:1042DC00AE07EEC39430400BEED394395005EE2468
:1042EC00D0FF22EEC39461400BEED394665005EEE2
:1042FC0024A9FF22EEC39441400BEED39446500503
:08430C00EE24C9FF22AF0622D6
:104455009062ADE004F070069062ACE004F090620A
:0A446500ACE0FEA3E0FF1243FF22CB
:100003001244551242DCEFC454F0FEC006124455AC
:080013001242DCD0E02FFF22B5
:1040B500E4906BE1F0124455906BE2EFF0C394305D
:1040C5004018E0FFD394395011906BE1E02405F5D9
:1040D50082E43461F583EFF08011906BE1E0240513
:1040E500F582E43461F583E4F0800C906BE1E00443
:1040F500F0E0D3940840BE75310075320075330089
:0C410500E4F5347B017A617905122A4848
:01411100228B
:043D63008E2B8F2CE8
:103D67009062ACE4F0A374FFF0124455EF606EF478
:103D7700606B852C82852B83E493B507EC752D0149
:103D8700E52C252DF582E4352BF583E4936025900A
:103D970062ADE0252DFF9062ACE03400FE1243FFD8
:103DA700E52C252DF582E4352BF583E493B507043F
:103DB700052D80CCE52C252DF582E4352BF583E404
:103DC7009370A6E52D24FFFFE434FFFE9062ADE07B
:103DD7002FF09062ACE03EF07E007F0122E4FEFF10
:013DE70022B9
:1035A2007E147F8A123D63EF4E70037F01227E14E8
:1035B2007F8D123D63EF4E600C124455EF24D024F0
:1035C200FF920F8002D20F7E147F93123D63EF4E63
:1035D200600C124455EF24D0906682F08005E4908E
:1035E2006682F07E147F99123D63EF4E600C1244A6
:1035F20055EF24D090668EF08005E490668EF07EC2
:10360200147F9F123D63EF4E600C124455EF24D09D
:1036120024FF92018002C2017E147FA5123D63EF56
:103622004E600C124455EF24D09062B4F08005E451
:103632009062B4F090633F63A20190667C63A20142
:103642007F061225E030013B7E147FAB123D63EF13
:103652004E603012000390667CEFF0120003906619
:103662007DEFF012000390667EEFF0120003906689
:103672007FEFF0120003906680EFF0120003906675
:0636820081EFF07F002241
:10422100906577E0C3947C40027F0A906577E0FE59
:1042310004F074B52EF582E43462F583EFF0BF0A21
:1042410027906577E0FF04F074B52FF582E43462BE
:10425100F583E4F0906577E0FF123DE890657774AF
:0942610008F09062B6E004F022BE
:10416E009080007480F090633763A201F583F5822E
:10417E0063A2017F081225E090633F63A201908045
:10418E008863A2017F0A1225E09080927407F0A343
:10419E0074D0F0A37406F0906349E0FF9080B1F004
:1041AE009080E1EFF09080957455F0A3F090800030
:0A41BE007401F090800974F0F02203
:103FE900908009E04410F09080A0E070609080A17A
:103FF9007482F09080A874FFF0A3F0A3F0A3F07F7F
:10400900039080AEEFF0A374CBF09080007402F0BF
:10401900906BCF12237E00000000906BCFE0908060
:1040290040F0906BD0E0908041F0906BD1E09080AF
:1040390042F0906BD2E0908043F0A3E4F0A3F0A3A8
:0D404900F0A3F0908018F0A3F0A3F0A3F016
:014056002247
:10411200908009E04440F09080D17482F07F039057
:1041220080DEEFF0A374CCF09080027402F0906B0A
:10413200D312237E00000000906BD3E0908058F0F1
:10414200906BD4E0908059F0906BD5E090805AF05B
:10415200906BD6E090805BF0A3E4F0A3F0A3F0A311
:0B416200F0908030F0A3F0A3F0A3F079
:01416D00222F
:103F6F00908009E04420F09080B8E0706C9080B9A8
:103F7F007482F07F039080C6EFF07FCDA3EFF07FC8
:103F8F00039080C4EFF0A374CDF09080C074FFF065
:103F9F00A3F0A3F0A3F09080017402F0906BD712FE
:103FAF00237E00000000906BD7E090804CF0906B68
:103FBF00D8E090804DF0906BD9E090804EF0906BF0
:103FCF00DAE090804FF0A3E4F0A3F0A3F0A3F09019
:093FDF008024F0A3F0A3F0A3F08C
:013FE80022B6
:103E6D008C268D27A907EAFDE975F018A424ACFF6F
:103E7D00E5F034808F82F583EDF0EBFDE975F018F8
:103E8D00A4FFAEF024ACFBEE34808B82F583A3ED62
:103E9D00F08527828C83E0FDEF24A8FFEE3480FEB1
:103EAD008F82F583EDF08527828C83A3E08F828E40
:103EBD0083A3F0852782852683A3A3E0FDE975F012
:103ECD0018A424A8FFE5F03480FE8F82F583A3A308
:103EDD00EDF08527828C83A3A3A3E08F828E83A32D
:043EED00A3A3F02279
:063C55008D2BAB07AA064F
:103C5B00908000E030E5079065797401F022906B5D
:103C6B00CFE0FCA3E0FDA3E0FEA3E0F52F8E2E8DAD
:103C7B002D8C2CAE02AF038E838F8263A201E52EB7
:103C8B00540744C0F583852F8263A201AF2B122604
:103C9B0052E4FCFDFEE52F252BF52FEE352EF52EF0
:103CAB00ED352DF52DEC352CF52C908040E52CF0D9
:103CBB00A3E52DF0A3E52EF0A3E52FF09080007483
:103CCB0020F0AF2FAE2EAD2DAC2C906BCF122372FC
:013CDB0022C6
:063CDC008D26AB07AA06CD
:103CE200908002E030E5079065797403F022906BD2
:103CF200D3E0FCA3E0FDA3E0FEA3E0F52A8E298D2C
:103D0200288C27AE02AF038E838F8263A201E5293E
:103D1200540744D0F583852A8263A201AF26122676
:103D220052E4FCFDFEE52A2526F52AEE3529F52981
:103D3200ED3528F528EC3527F527908058E527F052
:103D4200A3E528F0A3E529F0A3E52AF09080027408
:103D520020F0AF2AAE29AD28AC27906BD312237284
:013D6200223E
:023A89008F2686
:103A8B00908001E030E5099065797402F07F0022A7
:103A9B00906BD7E0FCA3E0FDA3E0FEA3E0F52A8E3C
:103AAB00298D288C2790667C63A201E52954074455
:103ABB00C8F583852A8263A2017F06122668E52A50
:103ACB002406F52AE43529F529E43528F528E435CB
:103ADB0027F52790657A63A201E529540744C8F5B9
:103AEB0083852A8263A201AF26122668E4FCFDFEC1
:103AFB00E52A2526F52AEE3529F529ED3528F52871
:103B0B00EC3527F52790804CE527F0A3E528F0A3AB
:103B1B00E529F0A3E52AF09080017420F0AF2AAEDE
:0D3B2B0029AD28AC27906BD7122372AF266E
:013B3800226A
:1032C1009081E0E0F526052605260526052605263A
:1032D10005260526052605260526908010E0F529F8
:1032E100A3E0F52AA3E0F52BA3E0F52C9081E1E022
:1032F100F526052605260526052605260526052685
:10330100052605260526908014E0F52DA3E0F52E6F
:10331100A3E0F52FA3E0F530E52FB52B08E530B597
:103321002C037F0022E4F526E52F540744E0F583C2
:1033310085308263A20190637663A2017F08122621
:103341009890637863A2019062AE63A2017F061236
:1033510025E0906376E0F527A3E0F528E4F52690D3
:103361006376E0702AA3E024F8F526E52F5407449C
:10337100E0F58385308274082582F582E43583F592
:103381008363A20190637663A201AF26122698AEF1
:1033910027E4FCFDE5302528F530E52F3EF52FED3E
:1033A100352EF52EEC352DF52D908014E52DF0A35D
:1033B100E52EF0A3E52FF0A3E530F09080007440F6
:0333C100F0AF2644
:0133C40022E6
:102BEC009081E6E0F5260526052605260526052610
:102BFC0005260526052605260526908028E0F529BC
:102C0C00A3E0F52AA3E0F52BA3E0F52C9081E7E0F7
:102C1C00F526052605260526052605260526052660
:102C2C0005260526052690802CE0F52DA3E0F52E33
:102C3C00A3E0F52FA3E0F530E4F526E52FB52B0A3C
:102C4C00E530B52C05C208022D58E52F540744F089
:102C5C00F58385308263A20190637663A2017F08BD
:102C6C00122698906376E0F527A3E0F528E5284531
:102C7C002770099080027410F07F0022906683E028
:102C8C00FFF46030906378E06F6003022D1F906654
:102C9C0084E0FF906379E06F7079906685E0FF9037
:102CAC00637AE06F706D906686E0FF90637BE06FF7
:102CBC006031805F906378E0906683F0906379E098
:102CCC00906684F090637AE0906685F090637BE088
:102CDC00906686F090637CE0FFA3E090634ACFF0AF
:102CEC00A3EFF0906376E0702AA3E024F8F526E5D4
:102CFC002F540744F0F58385308274082582F582C1
:102D0C00E43583F58363A20190637663A201AF2659
:102D1C00122698AE27E4FCFDE5302528F530E52F8A
:102D2C003EF52FED352EF52EEC352DF52DAF2CAEC9
:102D3C002BAD2AAC29AB30AA2FA92EA82DD3122348
:102D4C006140099080027410F07F002290802CE585
:102D5C002DF0A3E52EF0A3E52FF0A3E530F0908045
:062D6C00027440F0AF26E6
:012D7200223E
:102D73009081E3E0F526052605260526052605268A
:102D83000526052605260526052690801CE0F5293F
:102D9300A3E0F52AA3E0F52BA3E0F52C9081E4E072
:102DA300F5260526052605260526052605260526D8
:102DB300052605260526908020E0F52DA3E0F52EB7
:102DC300A3E0F52FA3E0F530E4F526E52FB52B0AB4
:102DD300E530B52C05C209022EC9E52F540744E896
:102DE300F58385308263A20190600463A2017F0EA4
:102DF3001226AE906004E0F527A3E0F52890600C5E
:102E0300E0FFF4604A90667CE0FEEF6E7079A3E029
:102E1300FF90600DE06F706F90667EE0FF90600E34
:102E2300E06F706390667FE0FF90600FE06F705714
:102E3300906680E0FF906010E06F704B906681E0D9
:102E4300FF906011E06F703FE4906013F080089092
:102E5300601374FFF0D2D9906004E0702AA3E024D9
:102E6300F2F526E52F540744E8F583853082740E86
:102E73002582F582E43583F58363A20190600463C0
:102E8300A201AF261226AEAE27E4FCFDE5302528CD
:102E9300F530E52F3EF52FED352EF52EEC352DF5DE
:102EA3002DAF2CAE2BAD2AAC29AB30AA2FA92EA85F
:102EB3002DD31223615006E5284527700990800120
:102EC3007410F07F0022908020E52DF0A3E52EF012
:102ED300A3E52FF0A3E530F09080017440F0AF2616
:012EE30022CC
:0434BA008E2B8F2C9A
:1034BE00908000E030E5079065797401F022906B02
:1034CE00CFE0FCA3E0FDA3E0FEA3E0F5328E318D4C
:1034DE00308C2FE532FFE5315407FEE42FF52EEE4A
:1034EE0034C0F52D852E82F5837423F0052EE52E3E
:1034FE007002052D532DC7F582852D83740AF005B4
:10350E002EE52E7002052D532DC790633F63A20149
:10351E00852D83852E8263A2017F061226527406A4
:10352E00252EF52EE4352DF52D852B83852C8263E6
:10353E00A201852D83852E8263A201122636E4FC1C
:10354E00FDFE906BCFE0F8A3E0F9A3E0FAA3E02F25
:10355E00FFEE3AFEED39FDEC38FCEF2408FFE43EB9
:10356E00FEE43DFDE43CFC906BCF122372906BCFDA
:10357E00E0908040F0906BD0E0908041F0906BD165
:10358E00E0908042F0906BD2E0908043F09080000B
:03359E007420F0A6
:0135A1002207
:0A31BA008E2B8F2C8C2D8D2E8B2F69
:1031C400908000E030E5079065797401F022906BFF
:1031D400CFE0FCA3E0FDA3E0FEA3E0F5358E348D43
:1031E400338C32E535FFE5345407FEE42FF531EE38
:1031F40034C0F530853182F5837423F00531E5312F
:10320400700205305330C7F582853083740AF005A7
:1032140031E531700205305330C790633F63A2013A
:1032240085308385318263A2017F0612265274069B
:103234002531F531E43530F530852B83852C8263D7
:10324400A20185308385318263A2011226368F362E
:10325400EF2531F531E43530F530E52F6017852D54
:1032640083852E8263A20185308385318263A20126
:10327400AF2F122652E5362408252FF52FFFE4FC44
:10328400FDFEE5352FF535EE3534F534ED3533F502
:1032940033EC3532F532908040E532F0A3E533F07B
:1032A400A3E534F0A3E535F09080007420F0AF3549
:0C32B400AE34AD33AC32906BCF122372FD
:0132C00022EB
:063769008E288F298D2A35
:10376F00908000E030E5079065797401F022906B4E
:10377F00CFE0FCA3E0FDA3E0FEA3E0F5308E2F8D9C
:10378F002E8C2DE530FFE52F5407FEE42FF52CEEA0
:10379F0034C0F52B852C82F5837423F0052CE52C92
:1037AF007002052B532BC7F582852B83EBF0052C6D
:1037BF00E52C7002052B532BC790633F63A2018545
:1037CF002B83852C8263A2017F0612265274062555
:1037DF002CF52CE4352BF52B85288385298263A2C4
:1037EF0001852B83852C8263A201AF2A1226527486
:1037FF0008252AF52AFFE4FCFDFEE5302FF530EE13
:10380F00352FF52FED352EF52EEC352DF52D90802E
:10381F0040E52DF0A3E52EF0A3E52FF0A3E530F062
:10382F009080007420F0AF30AE2FAD2EAC2D906B8A
:04383F00CF1223720F
:013843002262
:023DE8008F3F0B
:103DEA00908000E030E5079065797401F022906BCD
:103DFA00CFE0FCA3E0FDA3E0FEA3E0F5438E428DF5
:103E0A00418C40E543FFE5425407FEE42FFFEE34C0
:103E1A00C09062B563A201F5838F8263A201AF3FAE
:103E2A00122652E4FCFDFEE543253FF543EE3542FA
:103E3A00F542ED3541F541EC3540F540908040E5DD
:103E4A0040F0A3E541F0A3E542F0A3E543F09080FA
:103E5A00007420F0AF43AE42AD41AC40906BCF123C
:023E6A002372C1
:013E6C002233
:063688008E2E8F2FAB0512
:10368E00908000E030E5079065797401F022906B30
:10369E00CFE0FCA3E0FDA3E0FEA3E0F5358E348D74
:1036AE00338C32E535FFE5345407FEE42FF531EE69
:1036BE0034C0F530853182F5837423F00531E53160
:1036CE00700205305330C7F582853083EBF005313B
:1036DE00E5317002053090633F63A201853083852A
:1036EE00318263A2017F0612265274062531F5310E
:1036FE00E43530F5305330C7E52E85318285308381
:10370E00F00531E531700205305330C7F582853052
:10371E0083E52FF00531E531700205305330C7E5F2
:10372E0035240AF535E43534F534E43533F533E430
:10373E003532F532908040E532F0A3E533F0A3E563
:10374E0034F0A3E535F09080007420F0AF35AE3440
:0A375E00AD33AC32906BCF12237232
:01376800223E
:0A44B400E4FEEEC39F50030E80F8F3
:0144BE0022DB
:1043FF00A2AF921EC2AF438E2075D2028F828E83E0
:0C440F00E0FFE4F5D2538EDFA21E92AF56
:01441B00227E
:10436F00E5D220E0FBA2AF921EC2AF43D2028F82F2
:10437F008E83EDF075D25063D250A21E92AFE5D26C
:03438F0020E0FB30
:014392002208
:103EF100E4FDED2401FFE433FE1243FF74372DF599
:103F010082E43463F583EFF00DBD3FE6E4FDED247B
:103F11007FFFE433FE1243FF742D2DF582E43461FB
:103F2100F583EFF0742D2DF582E43461F583E070B3
:103F31001B742D2DF582E43461F5837420F0742E09
:103F41002DF582E43461F583E4F080040DBD80BE7B
:103F5100E49061ACF0FDEDFF7E001243FF74AD2DE6
:0D3F6100F582E43461F583EFF00DBDFEE95B
:013F6E002230
:024314008B2BF1
:10431600A2AF921EC2AF85A22C53A2FE8E838F82BD
:1043260005A28C838D8274091226DCE52B53A2FE2E
:1043360043A2201226DE53A2DF852CA2A21E92AF34
:01434600FF77
:014347002253
:10441C00A2AF921EC2AF8C838D82EF1226DC43A218
:0C442C00201226DE53A2DFA21E92AFFF7A
:014438002261
:024393008F2673
:10439500A2AF921EC2AFE4F5838D8274061226DCAD
:1043A500E52643A2201226DE53A2DFA21E92AF7F8E
:0143B5000106
:0143B60022E4
:0243B7008F264F
:1043B900A2AF921EC2AFE4F5838D82740A1226DC85
:1043C900E52643A2201226DE53A2DFA21E92AF7F6A
:0143D90001E2
:0143DA0022C0
:10250500A907E7FFA805EF93C3966008403B74FC55
:102515002FFF80F00F08EF93C3966008402B74FBE4
:102525002FFF80E00F08EF93C3966008401B74FAF5
:102535002FFF80D00F08EF93D3966008400B74F9F6
:102545002FFF80C01F1F1F1F1FEF54FEF80303F747
:10255500E893FC08E893FD08E893FE08E893FF225A
:1025650009E993C39D6008402974FB29F980F109A5
:10257500E993C39E6008401A74FA29F980E209E9D3
:1025850093D39F6008400B74F929F980D319191961
:102595001919E9C313C313FF22740093F8ECC39808
:1025A5004024701F740193F8EDC39840197014749A
:0E25B5000293F8EEC398400E7009740393F879
:1025C300EFC39840037F00227F0122EDF8E6F00875
:1025D300A3DFFA22EDF8E0F608A3DFFA22E0A36313
:1025E300A201F0A363A201DFF475A2002263A2019A
:1025F300F0A363A20122E0A363A201F0A363A201FB
:10260300E0A363A201F0A363A201E463A201F0A328
:1026130063A201DFE175A20022E0A363A2016DFEC4
:10262300936CFDEE058393FC158363A201DFEA75CA
:10263300A200227F00E493A363A201F00F600CA326
:10264300E583C2E3F58363A20180EA75A20022E079
:10265300A363A201F0A3E583C2E3F58363A201DFD1
:10266300EE75A20022E0A363A201F0A3E583C2E416
:10267300D2E3F58363A201DFEC75A20022E0A3633A
:10268300A201F0A3E58344F8C2E5F58363A201DF69
:10269300EC75A20022E583C2E3F583E0A363A20104
:1026A300F0A363A201DFEE75A20022E583C2E4D2A8
:0A26B300E3F583E0A363A201F0A3A6
:1026BD0063A201DFEC75A20022E58344F8F583E007
:1026CD00A363A201F0A363A201DFEE75A20022F9BC
:1026DD0022C002C004C00612FFF0D006D004D00202
:0126ED0022CA
:10001E00BF360BD217E4F545F546F561F562BF37ED
:04002E0002C21722D1
:10405700C2A9438902906BCAE0FFF58C8F8A75D994
:104067000475DA4875DB3175DC4975DD4975DE3174
:10407700E4F5E9F5F9F5EBF5FB906BC8E06016752B
:10408700EC1075ED10E4F5FCF5FD755D08755B103A
:10409700755C01801375EC8075ED80E4F5FCF5FD2A
:0E40A700755D80F55B755C10E4F5EEF5FE22AC
:0E44A500E4FFD28C75D84075B740D2AED2AFCE
:0144B30022E6
:03003300022EE4B6
:0B2EE400C0E0C083C082C0D075D008E1
:102EEF00C2AF30DC56C3E5EC95EEC3955D5012E5ED
:102EFF005C25ECF5EC30D70405FC801685FCFC80D6
:102F0F0011C3E5EC955CF5EC30D70415FC80038517
:102F1F00FCFC301724854682854583E590F00546F5
:102F2F00E54670020545F582854583E5EEF00546D9
:102F3F00E5467002054553450FC2DC30D9293017DD
:102F4F0024854682854583E590F00546E546700267
:102F5F000545F582854583E5EBF00546E5467002AC
:102F6F00054553450FC2D930DA5DE55B700405FCAA
:102F7F008010E55B25ECF5EC30D70405FC8003856C
:102F8F00FCFC301840E5475480F544E54725E0F553
:102F9F0047309702054720160363470130270FE597
:102FAF0047B56321755900755E00C2278017055E0E
:102FBF00E55E5407700F535E3FE55E131313541F06
:102FCF002449F8A647C2DA30DB71E55B700405FDD2
:102FDF008010E55B25EDF5ED30D70405FD80038509
:102FEF00FDFDE55F655A6029E55A54077013E55AF0
:102FFF00131313541F2451F8E6F5482014036348A4
:10300F00FFE548339296E54825E0F548055A535AAF
:10301F003FB292301723854682854583E590F005B0
:10302F0046E54670020545F582854583E4F0054681
:0D303F00E5467002054553450FC2DBD2AFD8
:09304C00D0D0D082D083D0E03254
:101BD9004241554400575F4D4F44454D00494E56CB
:101BE9005F52454300494E565F5452414E53004996
:101BF9004E565F414C4C004D4150424F41524400BA
:101C0900554E49544D00003E2A2C312CCFE0F0E0CE
:101C1900ECE5F2F0FB20F1E8EDF5F0EEEDEDEEE3A9
:101C2900EE20EFEEF0F2E00A003E4C2C4230312C6F
:101C3900256C752CD1EAEEF0EEF1F2FC20EEE1EC28
:101C4900E5EDE02C35302C3130302C3230302C336E
:101C590030302C3630302C313230302C3234303078
:101C69002C343830300A003E422C4731302C256262
:101C7900752CC8EDE2E5F0F1E8FF20EDE020EFF08A
:101C8900E8B8ECE50A003E422C4731312C25627553
:101C99002CC8EDE2E5F0F1E8FF20EDE020EFE5F0FA
:101CA900E5E4E0F7E50A003E422C4730322C256294
:101CB900752CD3EFF0E0E2EBE5EDE8E520EFEEF28D
:101CC900EEEAEEEC2020285254532D435453290AAE
:101CD900003E532C4730332C256C752CC7E0E4E5C6
:101CE900F0E6EAE020F1F2E0F0F2E020EFE5F0E5DD
:101CF900E4E0F7E828ECF1290A003E532C47303399
:101D09002C256C752C202AE7E0E4E5F0E6EAE020D2
:101D1900F1F2E0F0F2E020EFE5F0E5E4E0F7E828A1
:101D2900ECF1290A003E2A2C312CCCEEF1F2EEE23C
:101D3900EEE920EAEEEDF2F0EEEBEBE5F020CACFAA
:101D49002022C8F1E5F2FC222E20CFF0EEF2EEEAD5
:101D5900EEEB20D2CC3531320A003E532C473137D5
:101D69002C25732CD0E5E2E5F0F1E8E2EDFBE52066
:101D7900D2C8D20A003C21003C4230313D003C47E8
:101D890031303D003C4731313D003C4730323D0068
:101D99003C4730333D003C4731373D000ACDE5E84B
:101DA900E7E2E5F1F2EDFBE920EFE0EAE5F2202DCB
:101DB90020000ACFF0E8EDFFF220F6E8EAEBE8F7B9
:101DC900E5F1EAE8E920EFE0EAE5F220D2D12000E6
:101DD900202D20EEF8E8E1EAE020E4EBE8EDFB2134
:101DE9000A00202D20EEF8E8E1EAE020EDEEECE52E
:101DF900F0E020E1EBEEEAE0210A00202D20EEEAF6
:101E0900210A000ACFF0E8EDFFF220D2D120F1EE4D
:101E190020E2F0E5ECE5EDE5EC20000ACFF0E8ED95
:101E2900FFF220EFE0EAE5F220F120D2C8D220ED5E
:101E3900EEECE5F0EEEC202D20000ACEF8E8E1EA20
:101E4900E020E4E0EDEDFBF5210A000ACEF8E8E137
:101E5900EAE020F1E8EDF5F0EEEDE8E7E0F6E8E894
:101E69000A000AD6E8EAEB20D2C8D20A000AD6E864
:101E7900EAEB20D2D10A000A2E2E2EE020E4EEEB66
:101E8900E6E5ED20E1FBF2FC20D2C8D2210A000AE6
:101E99002E2E2EE020E4EEEBE6E5ED20E1FBF2FC50
:101EA90020D2D1210A000ACFE5F0E5E4E0F7E020ED
:101EB900E7E0EAEEEDF7E8EBE0F1FC0A000AC3EE31
:101EC900F2EEE220EFE0EAE5F220EA20EEF2EFF0AE
:101ED900E0E2EAE50A00FF1BD9FF1BDEFF1BE6FF74
:101EE9001BEEFF1BF8FF1C00FF1C09FF1C0F00085D
:0E1EF900040C020A060E0109050D030B070F6B
:10443F005266900000000000000000000000000025
:05444F00000000000068
:10446F00EF540F901EF793FEC454F0FEEFC4540F99
:04447F00932EFF2257
:0241C8008F2E38
:1041CA00906AB7E0FF04F074232FF582E43468F5AF
:1041DA00837420F0E4FFEFC39D503BE52E75F00396
:1041EA00A424DFF582E4341EF583E493FB7401937F
:1041FA00FA740293F98F82758300122222FE906A62
:10420A00B7E02423F582E43468F583EEF00F906A70
:06421A00B7E004F080C0D3
:01422000227B
:10434800742D2FF582E43461F583E0FE6420601655
:10435800906AB7E0FD04F074232DF582E43468F523
:0643680083EEF00F80DA85
:01436E00222C
:1026EE00200B09AF267E007D03123688E4906AB770
:1026FE00F0F526E52675F003A424DFF582E4341EFA
:10270E00F583E493FB740193FA740293F912220990
:10271E00700302289AE4F528F529F527742D25274C
:10272E00F582E43461F583E0FF7003022895E52617
:10273E0075F003A424DFF582E4341EF583E493FBE5
:10274E00740193FA740293F985288275830012221C
:10275E0022FEEFB506087529010528022890E52905
:10276E007003022890EE600302288BAD28AF26126C
:10277E0041C8E526B407004003022895902791F83A
:10278E002828730227A602284002287502287902FB
:10279E00287D022883022887AF27124348742D25EF
:1027AE0027F9E43461FA7B01C0031B8B31753200CB
:1027BE00753300E4F534D003122A488F2D8E2C8DFC
:1027CE002B8C2AE4FFFEFDFCAB2DAA2CA92BA82AEC
:1027DE00C31223616022AB2DAA2CA92BA82AE47F59
:1027EE00207E1CFDFC1222C1122353906BC9EEF009
:1027FE00A3EFF0E4906BC8F0E47FB07E04FDFCAB79
:10280E002DAA2CA92BA82AD3122361407A906BC82B
:10281E007401F0AB2DAA2CA92BA82A7F007EC2FD35
:10282E007C001222C1122353906BC9EEF0A3EFF07D
:10283E008055AF27124348D21A742D2527F9E43458
:10284E0061FA7B01C0031B8B31753200753300E4D6
:10285E00F534D003122A488F2D8E2C8D2B8C2A9076
:10286E0066A2E52DF08020D216801CD2148018D2DC
:10287E0016D2148012D215800ED210800AE4F529D9
:0C288E00F528052702272A05260227014D
:01289A00221B
:1033C5007BFF7A1C79101218DF906BC8E0602FA381
:1033D500E0FEA3E0FFC3E49FFFE49EFEAB07FAE433
:1033E500F9F8FF7EC27D01FC1222C18F318E308D2E
:1033F5002F8C2E7BFF7A1C79321218DF802F906B71
:10340500C9E0FEA3E0FFC3E49FFFE49EFEAB07FA1D
:10341500E4F9F87F207E1CFDFC1222C18F318E302D
:103425008D2F8C2E7BFF7A1C79321218DF7BFF7A69
:103435001C7970A216E433F52E1218DF7BFF7A1C77
:10344500798FA214E433F52E1218DF7BFF7A1C79ED
:10345500B0A21AE433F52E1218DF301A1F7BFF7A5B
:103465001C79DA9066A2E075F00AA4FFAEF0E48F4D
:10347500318E30F52FF52E1218DF801D7BFF7A1D5A
:1034850079039066A2E075F00AA4FFAEF0E48F31EF
:103495008E30F52FF52E1218DF7BFF7A1D792E124F
:1034A50018DF752E01752F677530A37BFF7A1D799F
:0534B500631218DF2284
:10289B007E1D7F7E123D63EF4E70037F01227E1DF6
:1028AB007F81123D63EF4E70030229421240B590B7
:1028BB006BDD122372E4FFFEFDFC906BDDE0F8A3F1
:1028CB00E0F9A3E0FAA3E0FBC31223616025906B50
:1028DB00DDE0F8A3E0A3E0A3E0E47F207E1CFDFC99
:1028EB001222C1122353906BC9EEF0A3EFF0E490C8
:1028FB006BC8F0E47FB07E04FDFC906BDDE0F8A3C9
:10290B00E0F9A3E0FAA3E0FBD31223614038906B0C
:10291B00C87401F0906BDDE0F8A3E0A3E0A3E07FC7
:10292B00007EC27D017C001222C1122353906BC921
:10293B00EEF0A3EFF0800F906BC974FFF0A374B8A7
:10294B00F0E4906BC8F07E1D7F87123D63EF4E6005
:10295B000C124455EF24D024FF92168002C2167E2F
:10296B001D7F8D123D63EF4E600C124455EF24D04A
:10297B0024FF92148002C2147E1D7F93123D63EFDD
:10298B004E600C124455EF24D024FF921A8002C2E1
:10299B001A7E1D7F99123D63EF4E60131240B5E412
:1029AB007B0AFAF9F81222C19066A2EFF08005E4D7
:1029BB009066A2F07E1D7F9F123D63EF4E6058E440
:1029CB00906BDBF0124455906BDCEFF0643C60478E
:1029DB00906BDCE0FF906BDBE0FE04F074A32EF554
:1029EB0082E43467F583EFF0124455906BDCEFF023
:1029FB00643C6009906BDBE0C3948040D3906BDB4D
:102A0B00E0B4800214F0906BDBE024A3F582E43495
:102A1B0067F583E4F08023906BDBE0FF04F074A395
:102A2B002FF582E43467F5837420F0906BDBE024A0
:0C2A3B00A3F582E43467F583E4F07F002B
:012A4700226C
:1043DB00906BC974FFF0A374B8F0E4906BC8F01243
:1043EB00289BEF60031226EEE4F55FF55A12405757
:0443FB001230552205
:1030550075637FC213D218C21DD227C21BC211C20B
:103065001CE4906963F0906AB6F0F526E52625E044
:103075002474F582E4346AAF82F5168F17F583E47C
:10308500F0A3F00526E526B420E2E4F52674A32591
:1030950026F582E43466F5837401F00526E526708D
:1030A500ECF527F528F52674A32526F582E4346783
:1030B500F583E0FF7003023178E528C374809481BD
:1030C5004003023178EFB42004052680DA74A32585
:1030D50026F582E43467F583E0642D702D052674AA
:1030E500A32526F9E43467FA7B01C0031B8B3175F0
:1030F5003200753300E4F534D003122A488F27C314
:10310500E5279528F5270527802374A32526F9E4C7
:103115003467FA7B01C0031B8B31753200753300B0
:10312500E4F534D003122A488F28752701E527D303
:103135009400401974809481501374A22528F58257
:10314500E43466F583E4F00528152780E074A325AB
:1031550026F582E43467F583E0FF642070030230CE
:10316500ACEF642D70030230ACEF70030230AC0598
:103175002680DAE4F526E52625E024B8F582E43450
:103185006AAF82F5168F1774A32526F582E4346697
:10319500F583E070047F2080027F00851782851605
:1031A50083EFF0A3E4F00526E526B480C9C291C2F9
:0431B500901244A58B
:0131B90022F3
:021F0700AB0726
:101F0900906004E024BE700302220824FE601B24B2
:101F1900FC70030220EE8000200D030222087E1DC2
:101F29007FA57C607D041231BA22906005E054E3FC
:101F39002480700302204624606003022208906016
:101F490007E0600302220890600EE0FE90600DE059
:101F59007C002400FFEC3E906BDBF0A3EFF0300D2A
:101F69000D7E1D7FBB7C6B7DDB7B021231BA9060DD
:101F790008E064066012200D030222087E1D7FD945
:101F8900E4FBFDFC1231BA22906006E0D3940740CD
:101F990012200D030222087E1D7FEBE4FBFDFC12DB
:101FA90031BA22906006E025E025E0F52625E024F7
:101FB90074F582E4346AAF82F5168F17E4F5278544
:101FC9001782851683A3E0FF12446F74092527F54C
:101FD90082E43460F583E06F600A85178285168391
:101FE900E04440F0851782851683E04480F09060D4
:101FF90006E024B8F582E4346BF58374C8F07409FB
:102009002527F582E43460F583E0FF12446F8517D4
:1020190082851683A3EFF074022517F517E43516A8
:10202900F5160527E527C394044094200D030222E1
:10203900087E1E7F04E4FBFDFC1231BA2290600881
:10204900E064086003022208906006E0D394074028
:1020590003022208300D0D7E1E7F0C7C6B7DDB7B1D
:10206900021231BA906007E0FF547FFE1313135434
:102079001FFE906006E025E025E02EF52625E024E8
:1020890074F582E4346AAD82F5168D17EF5407F5BD
:10209900267527806010E526D394004009E52713AB
:1020A900F527152680F0906007E030E70D85178247
:1020B900851683A3E04527F080108517828516834E
:1020C900A3E0FFE527F4FEEF5EF0906006E024B898
:1020D900F582E4346BF58374C8F08517828516831D
:1020E900E044C0F022906007E0FF30E603022208D6
:1020F900906006E0FED3940340030222087528602D
:10210900752909EF547FFFEEC43354E02FF52625D6
:10211900E024B8F582E4346AAF82F5168F17300DE2
:1021290013906BDDE526F07E1E7F247C6B7DDD7BC5
:10213900011231BA906008E0FFC313F526E4F527D0
:10214900E527C3952640030221EE85298285288348
:10215900E0FB7A00A3E0FEE42BFBEA3EFAC3EB9432
:1021690078EA6480946C50047AEC7B78D3EB948899
:10217900EA6480949340047A137B888517828516D4
:1021890083E030E514EB2488FFEA3413FE7C007DFC
:102199002812224FA3EFF08017AF03AE0212448337
:1021A9007C007D1412224F851782851683A3EFF0D8
:1021B90074022529F529E43528F528906006E024DC
:1021C900C0F582E4346BF58374C8F08517828516EF
:1021D90083E04480F074022517F517E43516F516E7
:1021E900052702214975166A7517B885178285165C
:0F21F90083A374F3F0851782851683E04480F08A
:0122080022B3
:0244CA008F263B
:0144CC0022CD
:0344CD007F00224B
:10390E00906AB6E0FFC3942040030239CDEF25E064
:10391E002474F582E4346AAF82F5168F17F583E0CE
:10392E0020E7030239C40513E513AE127002051227
:10393E0014F5828E83747FF0906AB6E02481FF05C1
:10394E0013E513AC127002051214F5828C83EFF09E
:10395E00851382851283F030D003E0F4F00513E571
:10396E001370020512851782851683A3E0FF0513D7
:10397E00E513AC127002051214F5828C83EFF085FC
:10398E001782851683A3E06455851382851283F012
:10399E0020D012851782851683A3E0F46455851313
:1039AE0082851283F00513E51370020512906AB634
:1039BE00E004F07F0522906AB6E004F002390EE4CE
:0639CE00906AB6F0FF2232
:10384400906963E0FFC394104003023907EFC45446
:10385400F024B8F582E4346AAF82F5168F17F58345
:10386400E020E7030238FE851382851283747FF01B
:103874000513E51370020512906963E02451FF8576
:103884001382851283F00513E51370020512F58285
:10389400851283EFF030D003E0F4F0E4FF0513E584
:1038A4001370020512851782851683A3E08513829F
:1038B400851283F00513E5137002051285178285BE
:1038C4001683A3E06455851382851283F020D012F9
:1038D400851782851683A3E0F464558513828512C7
:1038E40083F074022517F517E43516F5160FBF0893
:1038F400AC906963E004F07F1322906963E004F004
:09390400023844E4906963F0FF0D
:01390D002297
:10426A00300D0B7E1E7F43E4FBFDFC1231BA9066D3
:10427A009AE0FCA3E0FDA3E0FEA3E0FFE4FAF9F86C
:10428A00EF2401FFEA3EFEE93DFDE83CFC90669A18
:09429A00122372A212B392122247
:1042A300300D0B7E1E7F54E4FBFDFC1231BA906689
:1042B3009AE0FCA3E0FDA3E0FEA3E0FFE4FAF9F833
:1042C300EF2401FFEA3EFEE93DFDE83CFC90669ADF
:0942D300122372A212B39212220E
:1014B10030172DC3E5469562FFE5459561FED3EFF3
:1014C1009440EE940040197B087D40AF62AE6112FA
:1014D1003769E5622440FFE43561540FF5618F629D
:1014E100200003021598C200E4F52674B82526F5FC
:1014F10082E4346BF583E0700302158D74B8252600
:10150100F582E4346BF583E014F074B82526F58296
:10151100E4346BF583E07074E526C394085036E536
:101521002675F008A42474F582E4346AAF82F516B6
:101531008F17E4F527E527C394045050851782855A
:101541001683E0543FF0052774022517F517E4359B
:1015510016F51680E075F040E526A424B8F582E57D
:10156100F03468AF82F5168F17E4F527E527C394A9
:10157100205019851782851683E0543FF0052774A2
:10158100022517F517E43516F51680E00526E52640
:10159100641060030214EC201960301341E55E54BD
:1015A1003865596027E55924085438F55913131340
:1015B100541F2449F8E6FF0511E511AC107002052E
:1015C1001014F5828C83EFF0151A80D1E51A6003AF
:1015D10002177ED227D219C213C29102177E302779
:1015E1000302177ED291D213751A04301203751AB1
:1015F1001275106975116402177E300D1F30120FBC
:101601007E1E7F6B7C697D647B121231BA800D7EF8
:101611001E7F767C697D647B041231BAC2199069A0
:1016210064E0F030D00FA3E0F4FF906964E06F60F4
:101631001412426A22906965E0FF906964E06F606C
:101641000412426A22906964E054F0FFBF50047FA3
:101651000880027F018F26A212E433FFE526B40140
:10166100047E0180027E00EE5F6012300D0B7E1E53
:101671007F80E4FBFDFC1231BA1242A32220120446
:101681007F0180027F00E526B408047E0180027E8E
:1016910000EE5F6012300D0B7E1E7F98E4FBFDFCB7
:1016A1001231BA1242A322E4F527E527C395265049
:1016B10061E52725E02466F582E43469F583E0F0ED
:1016C10020D025E52725E02467F582E43469F583F8
:1016D100E0F46455FFE52725E02466F582E43469EA
:1016E100F583E0B507248026E52725E02467F58208
:1016F100E43469F583E06455FFE52725E02466F5C8
:1017010082E43469F583E06F600412426A2205279E
:101711008098E4F527E5262401FFE433FEC3E5279D
:101721009FEE6480F87480985020E52725E02464BA
:10173100F582E43469F583E0FF74232527F582E41B
:101741003469F583EFF0052780CBD21D906692E0D6
:10175100FCA3E0FDA3E0FEA3E0FFE4FAF9F8EF2427
:1017610001FFEA3EFEE93DFDE83CFC906692122352
:1017710072E526B40103D38001C3921222201B0318
:1017810002180CE55F655A6048E55F24085438FF8C
:10179100E55A54386F60047E0180027E00E51B60CB
:1017A100047D0180027D00EE5D700302187C05134B
:1017B100E513AC127002051214F5828C83E0FEE58C
:1017C1005F131313541F2451F8A6068F5F151B8056
:1017D100B8C290300D0B7E1E7FAFE4FBFDFC1231D1
:1017E100BAC21BC211906696E0FCA3E0FDA3E0FE25
:1017F100A3E0FFE4FAF9F8EF2401FFEA3EFEE93D38
:10180100FDE83CFC90669612237222E4F51B7512EA
:10181100697513F412390E8F1BE51B700512390E11
:101821008F1B1238448F26E52670051238448F2607
:10183100E526251BF51B64187041300D0D7E1E7FBA
:10184100C67C697DF47B181231BA7512697513F47F
:101851000513E513AE127002051214F5828E83E0B2
:10186100FFE55F131313541F2451F8A607E55F2406
:0B187100085438F55F151BD21BD29005
:01187C002249
:0B44BF00301C05C21C7F01227F002280
:1039D400E4FF0F2405F582E43461F5837408F00FE5
:1039E40074052401F582E43461F583E4F07C667D9A
:1039F40095FEED1DAA0470011CF5828A83E0FBAAE2
:103A0400070F74052AF582E43461F583EBF00EBEEA
:103A140004E07C667D99E4FEED1DAA0470011CF5AA
:103A2400828A83E0FBAA070F74052AF582E43461D5
:103A3400F583EBF00EBE04E07C667D9DE4FEED1D97
:103A4400AA0470011CF5828A83E0FBAA070F74059F
:103A54002AF582E43461F583EBF00EBE04E07C6663
:103A64007DA1E4FEED1DAA0470011CF5828A83E0A9
:103A7400FBAA070F74052AF582E43461F583EBF0A1
:043A84000EBE04E08E
:013A8800221B
:0344D000C2AE2257
:103BD500020921E493A3F8E493A34003F68001F2DC
:103BE50008DFF48029E493A3F85407240CC8C333F1
:103BF500C4540F4420C8834004F456800146F6DFC0
:103C0500E4800B0102040810204080904439E47ED2
:103C1500019360BCA3FF543F30E509541FFEE493B4
:103C2500A360010ECF54C025E060A840B8E493A37B
:103C3500FAE493A3F8E493A3C8C582C8CAC583CAA6
:103C4500F0A3C8C582C8CAC583CADFE9DEE780BE5E
:014454000067
:10220900BB010689828A83E0225002E722BBFE02D3
:09221900E32289828A83E4932206
:10222200BB010CE58229F582E5833AF583E0225071
:1022320006E92582F8E622BBFE06E92582F8E222BB
:0D224200E58229F582E5833AF583E49322D5
:10224F00C2D5EC30E709B2D5E4C39DFDE49CFCEEAA
:10225F0030E715B2D5E4C39FFFE49EFE1223C1C33E
:10226F00E49DFDE49CFC80031223C130D507C3E439
:06227F009FFFE49EFE2219
:1022850075F008758200EF2FFFEE33FECD33CDCC10
:1022950033CCC58233C5829BED9AEC99E582984093
:1022A5000CF582EE9BFEED9AFDEC99FC0FD5F0D670
:1022B500E4CEFBE4CDFAE4CCF9A88222B800C1B99A
:1022C5000059BA002DEC8BF084CFCECDFCE5F0CBD8
:1022D500F97818EF2FFFEE33FEED33FDEC33FCEB11
:1022E50033FB10D703994004EB99FB0FD8E5E4F9CC
:1022F500FA227818EF2FFFEE33FEED33FDEC33FCB9
:10230500C933C910D7059BE99A4007EC9BFCE99AAC
:10231500F90FD8E0E4C9FAE4CCFB2275F010EF2FF1
:10232500FFEE33FEED33FDCC33CCC833C810D707F1
:102335009BEC9AE899400AED9BFDEC9AFCE899F82C
:0E2345000FD5F0DAE4CDFBE4CCFAE4C8F922BF
:0E235300C3E49FFFE49EFEE49DFDE49CFC229B
:10236100EB9FF5F0EA9E42F0E99D42F0E89C45F0D2
:012371002249
:0C237200ECF0A3EDF0A3EEF0A3EFF022DE
:10237E00A8828583F0D083D08212239512239512E2
:10238E002395122395E473E493A3C583C5F0C58307
:10239E00C8C582C8F0A3C583C5F0C583C8C582C8A9
:0123AE00220C
:10187D00E53A242EF8E6053A22782B302502782E0B
:10188D00E475F001122465022209201EEB7F2ED291
:10189D001E8018EF540F2490D43440D4FF30220B07
:1018AD00EF24BFB41A0050032461FFE53B6002151D
:1018BD003B053EE53E7002053D30250D782BE47568
:1018CD00F001122465EF0223AF0242217403D225E9
:1018DD008003E4C225F53A8B2B8A2C892DE4F53B48
:1018ED00F53DF53EE53B60077F201218B880F57594
:1018FD003CFFC21FC21EC220C221C223C224C22667
:10190D00121886FF700D3025057F001218C9AF3EE5
:10191D00AE3D22B4255FC2D5C222121886FF24D057
:10192D00B40A00501A75F00A783B30D50508B6FF99
:10193D000106C6A426F620D5047002D22180D92432
:10194D00CFB41A00EF5004C2E5D222021AC9D21F39
:10195D0080C6D21E80C0D22080BCD2D580BAD22300
:10196D0080B47F201218B82020077401B53B0040C9
:10197D00F112187DFF1218B80218F1D226D2248068
:10198D009512187DFB12187DFA12187DF94A4B70CD
:10199D0006799A7A1B7BFF20202EE53B602A7E007C
:1019AD008E8275830012222260060EEE653C70F069
:1019BD00C2D5EBC0E0EAC0E0E9C0E0EE121B10D0EA
:1019CD00E0F9D0E0FAD0E0FB122209FF60AAEBC0EB
:1019DD00E0EAC0E0E9C0E01218B8D0E02401F9D087
:1019ED00E03400FAD0E0FBE53C0460DCD53CD98066
:1019FD00877BFF7A1B790CD220809C79108002792D
:101A0D0008C224C2268008D2D5790A8004790AC278
:101A1D00D5E53C047002F53CE4FAFDFEFF12187D9D
:101A2D00FC7B08201F1312187DFD7B10301E0A123F
:101A3D00187DFE12187DFF7B20EC3382D592D55098
:101A4D0013C3E4301E069FFFE49EFEE4201F039D9A
:101A5D00FDE49CFCE4CBF8C21FEC700CCFCECDCCDA
:101A6D00E824F8F870F38017C3EF33FFEE33FEED83
:101A7D0033FDEC33FCEB33FB994002FB0FD8E9EB64
:101A8D00301F05F8D0E0C448B21FC0E00AEC4D4E3F
:101A9D004F78207B0070C2EAB53C0040BCC0E0121C
:101AAD001B12D0F0D0E0201F04C4C0E0C4B21FC090
:101ABD00F01218A1D0F0D5F0EB0218F11224C419D0
:101ACD008E531A0858195F4C195B421A0C4F1A1491
:0F1ADD00441A14491974431A1A5519FE4619FE72
:101AEC004519FE471BBA5019632D19672E198A2BFD
:101AFC00196B231988201BA32A192348000019826B
:101B0C003F3F3F00790AA2D5202114302309B91098
:101B1C00020404B9080104A2D520240250010420B7
:101B2C0020689220B53B005034C0E07F2030211952
:101B3C007F30A22072247223500F121B69C220C264
:101B4C0024C223C2267F30800F302303E9C0E01269
:101B5C0018B8302303D0E0F9D0E0B53BCC302317D4
:101B6C007F30B9100C1218B87F583022077F78805C
:101B7C0003B908031218B83020057F2D0218B87F5E
:101B8C00202026F87F2B2024F322922080CF286E51
:101B9C00756C6C2900D21F12187D301FF8C21F788B
:101BAC003B30D50108F60219232D50434958121821
:101BBC007D2403B405004001E4901BB5931218A9D1
:0D1BCC00743A1218A9D221753B04021A08C0
:10448300C3EE6480948040028007C3E49FFFE49EF0
:02449300FE2207
:102A48008B2E8A2F8930E4F53AF539F538F537F5C4
:102A580035F536E532453345316012EBC0E0EAC062
:102A6800E0E9C0E0AB31AA32A933122475AB2E05D8
:102A780030E530AA2F7002052F14F9122209F53B10
:102A8800C394094007E53BD3940D40E1E53B64203E
:102A980060DBE53BB42D054336038016E53BB42BDC
:102AA80005433601800C74FF2530F53074FF352F4F
:102AB800F52FE53460046410703FAB2EAA2FA930BF
:102AC80012220964306009E534702E75340A8029B1
:102AD800900001122222FF64786004EFB458134377
:102AE800360175341074022530F530E4352FF52F92
:102AF8008007E5347003753408AB2E0530E530AA3D
:102B08002F7002052F14F9122209F53BC394614076
:102B18000AE53BD3947A5003533BDF74D0253BF549
:102B28003BC3940A400CE53B9411406D74F9253B76
:102B3800F53BE53BD395345060433601853A3F85F4
:102B4800393E85383D85373CAF347E00E4FCFDAB2B
:102B58003AAA39A938A837122416C8ECC8C9EDC949
:102B6800CAEECACBEFCBE4FCFDFEEB253BF53AEE13
:102B78003AF539ED39F538EC38F537AF3AAE39ADC5
:102B880038FCAB3FAA3EA93DA83CD31223615003B1
:102B9800022B01433604022B01E53620E003E480D2
:102BA8002DE53245334531601EAB2EE53024FFF963
:102BB800E52F34FFFAEBC0E0EAC0E0E9C0E0AB3152
:102BC800AA32A933122475E53630E20774FFFFFEF6
:102BD800FDFC22E536AF3AAE39AD38AC3730E1030B
:042BE800022353224F
:1023AF00BB010689828A83F0225002F722BBFE010D
:0223BF00F32207
:1023C100BC000BBE0029EF8DF084FFADF022E4CC00
:1023D100F875F008EF2FFFEE33FEEC33FCEE9DECC9
:1023E100984005FCEE9DFE0FD5F0E9E4CEFD22ED0F
:1023F100F8F5F0EE8420D21CFEADF075F008EF2F59
:10240100FFED33FD4007985006D5F0F222C398FD49
:052411000FD5F0EA22E6
:10241600E88FF0A4CC8BF0A42CFCE98EF0A42CFC65
:102426008AF0EDA42CFCEA8EF0A4CDA8F08BF0A4E3
:102436002DCC3825F0FDE98FF0A42CCD35F0FCEB42
:102446008EF0A4FEA9F0EB8FF0A4CFC5F02ECD3907
:0F245600FEE43CFCEAA42DCE35F0FDE43CFC2274
:10246500FAE6FB0808E6F925F0F618E6CA3AF62278
:10247500BB011A89828A83D0F0D0E0F8D0E0F9D088
:10248500E0FAD0E0FBE8C0E0C0F00224F35016E922
:10249500F8D083D082D0E0F9D0E0FAD0E0FBC0825A
:1024A500C0830224EABBFE16E9F8D083D082D0E0CF
:0F24B500F9D0E0FAD0E0FBC082C0830224FC2201
:1024C400D083D082F8E4937012740193700DA3A3A7
:1024D40093F8740193F5828883E4737402936860BB
:0624E400EFA3A3A380DFBB
:0924EA00EBF608EAF608E9F62217
:0924F300EBF0A3EAF0A3E9F022EA
:0924FC00EBF208EAF208E9F22211
:00000001FF
